:100000000C9433010C9450010C9450010C94500149
:100010000C9450010C9450010C9450010C9450011C
:100020000C9450010C9450010C9450010C9450010C
:100030000C943B120C9450010C9450010C94500100
:100040000C9450010C94B0050C9450010C94501178
:100050000C94DA110C9450010C9450010C94500142
:100060000C9450010C9450010C9450010C945001CC
:100070004570692D4F5344205665722E302E392E0F
:10008000302E322E340000416B7475656C6C6573D4
:100090002053657474696E67000053657474696EEB
:1000A0006720200000486F6568656E73656E736F2A
:1000B000722000004853206D697420536368616C9E
:1000C00074657220000048656164696E6720486F3E
:1000D0006C642000004B6F6D706173732000004BE7
:1000E0006F6D70617373206669782000004750530C
:1000F00020416B74697620000041636873656E6B04
:100100006F7070656C756E67200000447265687270
:1001100061746520626567722E2000004665686C18
:1001200065722046433C2D3E4F5344200000556EDF
:100130007465727370616E6E756E672000004B653A
:10014000696E652053657474696E672D416E7A65BA
:10015000696765000050432F425420616B746976D3
:10016000000055656265726E65686D65204C65744A
:100170007A7465732053657474696E6700004B650B
:10018000696E65204465766976652D416E7A65698C
:100190006765000050432F425420616B74697600FC
:1001A0000055656265726E65686D65204C65747A90
:1001B0007465732044657669636500004F4E0000E6
:1001C0002D2D2D000044657669636520756E6420D1
:1001D00056657273696F6E736162667261676500FE
:1001E0000044656369766520202020203D200000C2
:1001F00046572D56657273696F6E203D200000468C
:100200004300004E43000046432D6F6C6420465768
:1002100000004550492D4D656E750050616C0050D1
:10022000432F4254004B656E6E756E670052432D2E
:1002300042657472696562000045786974004F4ECA
:10024000002D2D0076767D76767A76767E767677B8
:1002500076767B76767876767C76767976767D7627
:10026000767A76767E7611241FBECFEFD4E0DEBF9D
:10027000CDBF11E0A0E0B1E0ECE0F0E302C00590FA
:100280000D92A038B107D9F713E0A0E8B1E001C0A2
:100290001D92AC39B107E1F70E945D010C9404187E
:1002A0000C94000082E981BB8FE084BBAC9AAD9ACC
:1002B0008EE28ABBD99ADD9A08951092CE011092EF
:1002C000CA011092CF01E199FECF80E090E09FBB80
:1002D0008EBBE09A8DB380938701E199FECF81E0D8
:1002E00090E09FBB8EBBE09A8DB380930001E199B3
:1002F000FECF82E090E09FBB8EBBE09A8DB38093EF
:100300008801E199FECF87E190E09FBB8EBBE09A28
:100310008DB380939F01E199FECF88E190E09FBB70
:100320008EBBE09A8DB38093B801E199FECF8AE14C
:1003300090E09FBB8EBBE09A8DB380939003E199D0
:10034000FECF89E190E09FBB8EBBE09A8DB3809396
:10035000B4010E94C51582E981BB8FE084BBAC9AD1
:10036000AD9A8EE28ABBD99ADD9A0E94A905809146
:100370008701813019F40E944B1002C00E943B108B
:100380007894A89A0E94DF040E9412060E94FE0937
:100390008091B80185FF02C00E9482130E94400A2A
:1003A0000E941C118091B001813021F41092B001A3
:1003B0000E946216809182018130E9F410928201DC
:1003C0008091CE01882389F48091B401843069F44E
:1003D00080918701882349F480919401813029F428
:1003E00080E363E64AE00E94CA100E942E120E9437
:1003F00033120E949A13809185018130B9F5809162
:10040000CE01882399F5AA9A0E948D0E80919F01B2
:100410008823A9F40E9463090E947A0880918F03BF
:10042000882321F00E94A7120E94BD0A80918E03AA
:10043000882311F00E9415160E94940A16C080911C
:100440000201823054F00E94060A0E94A7120E9404
:10045000BD0A0E94D60B0E94940A8091020183304B
:1004600024F00E9463090E947A08AA988091800172
:100470008130A9F58091CE01882389F51092800101
:1004800080919F01882321F080910201833014F034
:100490000E946F0A80919C0190919D01019690931A
:1004A0009D0180939C010197CB9769F480919A01FB
:1004B00090919B01019690939B0180939A011092D9
:1004C0009D0110929C010E94480C0E948C0D80910D
:1004D0008D01813021F40E9410060E941106809146
:1004E0008101813009F05ECF8091CE01882309F02F
:1004F00059CF109281010E94060A80919F0181309C
:1005000009F050CF8091CE01882309F04BCF809124
:100510009E01813009F046CF10929E018091020128
:10052000813071F082301CF4882339F03BCF823067
:1005300081F0833009F036CF17C00E94B80A32CF5D
:100540000E948F0A84E064E00E94C1020E941306A8
:1005500029CF0E948F0A84E064E00E94C1020E94B9
:10056000FE090E94400A1ECF0E948F0A84E064E0C8
:100570000E94C1020E94FE090E94400A0E946F0A66
:1005800011CF782FD99827E030E041E050E0DB9898
:100590000000000000000000CA01022E02C0880F07
:1005A000991F0A94E2F7872311F0DA9A01C0DA98CA
:1005B0000000000000000000DB9A000000000000C6
:1005C0000000215030408FEF2F3F380701F727E020
:1005D00030E041E050E0DB98000000000000000047
:1005E000CA01022E02C0880F991F0A94E2F78623DF
:1005F00011F0DA9A01C0DA98000000000000000053
:10060000DB9A0000000000000000215030408FEF16
:100610002F3F380701F7DB98DA98D99A089584E0DC
:1006200064E00E94C10280E06CE40E94C10210926A
:100630008201809182018823E1F38CE66AE00E94C6
:10064000C10285E060E00E94C10208951F9380917D
:10065000B401823051F40E945B10109280018091AD
:1006600080018823E1F31092800182E661E74FEF79
:100670000E94CA101092800110E00DC08091850187
:10068000813011F40E948D0E80918001813019F427
:100690001092800111E08091BA01882311F4112396
:1006A00069F38091B401823011F40E94A2101123E9
:1006B00009F0E9C090917B03892F817080938F03AB
:1006C000892F887080938E03892F80728093910385
:1006D000892F84708093920380918B038093900381
:1006E0009093B8012091B801E199FECF88E190E0A4
:1006F0009FBB8EBB2DBB0FB6F894E29AE19A0FBE5A
:1007000020919003E199FECF8AE190E09FBB8EBBE0
:100710002DBB0FB6F894E29AE19A0FBE82E061E039
:1007200047E850E00E94C80D82E062E04AE950E0EC
:100730000E94C80D82E064E045EA50E00E94C80DC6
:1007400082E065E044EB50E00E94C80D82E066E084
:1007500046EC50E00E94C80D82E067E045ED50E0B5
:100760000E94C80D82E068E04FED50E00E94C80D85
:1007700082E069E04DEE50E00E94C80D82E06AE040
:1007800049EF50E00E94C80D82E06BE04EE251E07C
:100790000E94C80D4091B6015091B70184E162E01A
:1007A0000E949D0D8091B80180FF05C084E164E046
:1007B0004CEB51E004C084E164E040EC51E00E9465
:1007C000C80D8091B80181FF05C084E165E04CEB64
:1007D00051E004C084E165E040EC51E00E94C80DA6
:1007E0008091B80182FF05C084E166E04CEB51E0E6
:1007F00004C084E166E040EC51E00E94C80D8091A5
:10080000B80183FF05C084E167E04CEB51E004C010
:1008100084E167E040EC51E00E94C80D8091B8018E
:1008200084FF05C084E168E04CEB51E004C084E142
:1008300068E040EC51E00E94C80D8091B80185FF4E
:1008400005C084E169E04CEB51E004C084E169E05B
:1008500040EC51E00E94C80D8091B80186FF05C0B0
:1008600084E16AE04CEB51E004C084E16AE040ECD2
:1008700051E00E94C80D40918B0384E16BE050E091
:100880000E949D0D16C082E062E047E850E00E94A1
:10089000C80D82E065E04CE151E00E94C80DE1998D
:1008A000FECF88E190E09FBB8EBBE09A8DB3809332
:1008B000B8011F9108951F93809180018823E1F36F
:1008C0001092800183E666E740E00E94CA1010E0C3
:1008D0000DC080918501813011F40E94700E8091CD
:1008E0008001813019F41092800111E08091B501EE
:1008F000882311F4112369F3112309F054C082E015
:1009000062E045EC51E00E94C80D82E064E041EEF7
:1009100051E00E94C80D82E066E040EF51E00E9485
:10092000C80D8091B401813031F48EE064E04FEF66
:1009300051E00E94C80D8091B401823031F48EE004
:1009400064E043E052E00E94C80D8091B40184301D
:1009500031F48EE064E047E052E00E94C80D40911F
:100960003C038EE066E050E00E949D0D40913D0307
:1009700080E166E050E00E949D0D40913E0383E1DE
:1009800066E050E00E949D0D2091B401E199FECFF8
:1009900089E190E09FBB8EBB2DBB0FB6F894E29A25
:1009A000E19A0FBE0AC0E199FECF89E190E09FBBBA
:1009B0008EBBE09A8DB38093B4011F9108950E947D
:1009C0000F0383E66FE644E60E94CA10109280018E
:1009D000809180018823E1F387E062E040E750E006
:1009E0000E94C80D0E941306109280018091800120
:1009F0008823E1F310928001809180018823E1F344
:100A000010928001809180018823E1F3109280018F
:100A100084E064E00E94C10280E06CE40E94C102B4
:100A200080918701882319F40E945B041CC082E036
:100A300062E04EE751E00E94C80D82E064E044E9C4
:100A400051E00E94C80D82E066E041EA51E00E9458
:100A5000C80DE199FECF89E190E09FBB8EBBE09A83
:100A60008DB38093B401809180018823E1F31092CB
:100A70008001809180018823E1F31092800184E05D
:100A800064E00E94C10280E06CE40E94C102809197
:100A90008701882319F40E94260326C082E062E0C1
:100AA0004EE351E00E94C80D82E064E045E551E06C
:100AB0000E94C80D82E066E042E651E00E94C80D47
:100AC000E199FECF88E190E09FBB8EBBE09A8DB3A9
:100AD0008093B801E199FECF8AE190E09FBB8EBB85
:100AE000E09A8DB3809390038091B401823029F411
:100AF00083E66FE64AE00E94CA108091B40181301B
:100B000029F482E664E64AE00E94CA1080918001DE
:100B10008823E1F310928001809180018823E1F322
:100B200010928001809180018823E1F3109280016E
:100B3000809180018823E1F31092800180918001EF
:100B40008823E1F31092800184E064E00E94C102F6
:100B5000089582E083BF82E48EBD8AE089BF089554
:100B60001F920F920FB60F9211248F939F93809133
:100B700084018F5F8093840180918401883449F5DA
:100B800091E09093830110928401809194038F5F90
:100B90008093940380919403843631F410929403EB
:100BA000909380019093810180919403823319F492
:100BB00081E080938101809193038F5F8093930301
:100BC000809193038A3029F41092930381E08093FB
:100BD00082019F918F910F900FBE0F901F901895DB
:100BE000982F80538A3010F020E005C0903311F424
:100BF0002AE001C0282F892F81548A3110F4292F2F
:100C00002653892F81568A3110F4292F2C539D3277
:100C100011F429E403C09E3209F421E4822F0895DF
:100C200008950895089585E060E00E94C10286E07D
:100C300063E80E94C10287E060E90E94C10285E08A
:100C400060E00E94C10286E064E80E94C10287E081
:100C500061E90E94C10285E060E00E94C10286E075
:100C600065E80E94C10287E062E90E94C10285E056
:100C700060E00E94C10286E066E80E94C10287E04F
:100C800063E90E94C10285E060E00E94C10286E043
:100C900067E80E94C10287E064E90E94C10285E022
:100CA00060E00E94C10286E068E80E94C10287E01D
:100CB00065E90E94C10285E060E00E94C10286E011
:100CC00069E80E94C10287E066E90E94C10285E0EE
:100CD00060E00E94C10286E06AE80E94C10287E0EB
:100CE00067E90E94C10285E060E00E94C10286E0DF
:100CF00061EA0E94C10287E068E90E94C10285E0C2
:100D000060E00E94C10286E062EA0E94C10287E0C0
:100D100069E90E94C10285E060E00E94C10286E0AC
:100D200063EA0E94C10287E06AE90E94C10285E08D
:100D300060E00E94C10286E064EA0E94C10287E08E
:100D40006BE90E94C10285E060E00E94C10286E07A
:100D500065EA0E94C10287E06CE90E94C10285E059
:100D600060E00E94C10286E066EA0E94C10287E05C
:100D70006DE90E94C10285E060E00E94C10286E048
:100D800067EA0E94C10287E06EE90E94C10285E025
:100D900060E00E94C10286E068EA0E94C10287E02A
:100DA0006FE90E94C10285E060E00E94C10286E016
:100DB0006FEB0E94C10287E060EA0E94C10285E0F9
:100DC00060E00E94C10286E060EC0E94C10287E000
:100DD00061EA0E94C10285E060E00E94C10286E0F3
:100DE00061EC0E94C10287E062EA0E94C10285E0D4
:100DF00060E00E94C10286E062EC0E94C10287E0CE
:100E000063EA0E94C10285E060E00E94C10286E0C0
:100E100063EC0E94C10287E064EA0E94C10285E09F
:100E200060E00E94C10286E064EC0E94C10287E09B
:100E300065EA0E94C10285E060E00E94C10286E08E
:100E400065EC0E94C10287E066EA0E94C10285E06B
:100E500060E00E94C10286E066EC0E94C10287E069
:100E600067EA0E94C10285E060E00E94C10286E05C
:100E70006DED0E94C10287E068EA0E94C10285E030
:100E800060E00E94C10286E06EED0E94C10287E030
:100E900069EA0E94C10285E060E00E94C10286E02A
:100EA0006FED0E94C10287E06AEA0E94C10285E0FC
:100EB00060E00E94C10286E060EE0E94C10287E00D
:100EC0006BEA0E94C10285E060E00E94C10286E0F8
:100ED00061EE0E94C10287E06CEA0E94C10285E0D7
:100EE00060E00E94C10286E062EE0E94C10287E0DB
:100EF0006DEA0E94C10285E060E00E94C10286E0C6
:100F000063EE0E94C10287E06EEA0E94C10285E0A2
:100F100060E00E94C10286E064EE0E94C10287E0A8
:100F20006FEA0E94C10285E060E00E94C10286E093
:100F30006BEF0E94C10287E060EB0E94C10285E076
:100F400060E00E94C10286E06CEF0E94C10287E06F
:100F500061EB0E94C10285E060E00E94C10286E070
:100F60006DEF0E94C10287E062EB0E94C10285E042
:100F700060E00E94C10286E06EEF0E94C10287E03D
:100F800063EB0E94C10285E060E00E94C10286E03E
:100F90006FEF0E94C10287E064EB0E94C10285E00E
:100FA00061E00E94C10286E060E00E94C10287E029
:100FB00065EB0E94C10285E061E00E94C10286E00B
:100FC00061E00E94C10287E066EB0E94C1020895C1
:100FD000BF92CF92DF92EF92FF920F931F93CF9326
:100FE000DF937C01B62E8C0145E0C42ED12CC80EB7
:100FF000D91E862F90E0EC01CC0FDD1FC80FD91F42
:10100000C15FDE4F0EC085E0612F0E94C10286E005
:10101000602F0E94C10287E068810E94C1020F5FB9
:101020001F4F0C151D0578F38701065F1F4F8FE0DA
:1010300090E0E80EF91E8B2D90E0EC01CC0FDD1F47
:10104000C80FD91FC15FDE4F0EC085E0612F0E941F
:10105000C10286E0602F0E94C10287E068810E9481
:10106000C1020F5F1F4F0E151F0578F3DF91CF915F
:101070001F910F91FF90EF90DF90CF90BF90089558
:10108000EF92FF920F931F93CF93DF938C01EC01AC
:1010900055E0E52EF12CE80EF91E0DC085E06D2F10
:1010A0000E94C10286E06C2F0E94C10287E060E0CE
:1010B0000E94C1022196CE15DF0580F3E8012A9631
:1010C000015F1F4F0DC085E06D2F0E94C10286E0B9
:1010D0006C2F0E94C10287E060E00E94C10221964D
:1010E000C017D10780F3DF91CF911F910F91FF902F
:1010F000EF9008951F93CF93DF93E0913D02F0911D
:101100003E02F7FD1CC0CF016AE070E00E94F117BB
:10111000182F1695CF016AE070E00E94F11787E062
:1011200090E0861B9109EC0175E0CC0FDD1F7A95EC
:10113000E1F7880F991FC81BD90B279617C02227E4
:1011400033272E1B3F0BC9016AE070E00E94F117A4
:10115000182F16951C5FC9016AE070E00E94F11714
:101160008EE1689FE0011124C950DF4F80910B018F
:1011700090910C01C817D90739F080910B0190911B
:101180000C010E94400804C08091BD01811721F02C
:10119000CE01612F0E94E8071093BD01D0930C018E
:1011A000C0930B01DF91CF911F910895CF92DF92F1
:1011B000EF92FF920F931F93CF93DF938C01E62E54
:1011C00085E0612F0E94C10286E0602F0E94C1026B
:1011D000CE2CDD248DE291E0C80ED91E87E0F60109
:1011E00060810E94C102EEE1EE2EF12CE00EF11EB4
:1011F00085E06F2D0E94C10286E06E2D0E94C10223
:1012000087E0F60160810E94C102E801CC54DF4F03
:10121000025F1E4F85E06D2F0E94C10286E06C2F99
:101220000E94C10287E0F60160810E94C1026E96B1
:10123000C017D10779F7DF91CF911F910F91FF90E0
:10124000EF90DF90CF900895EF92FF920F931F934E
:10125000CF93DF937C0185E06F2D0E94C10286E071
:101260006E2D0E94C10287E060E00E94C1028701EA
:10127000025E1F4F85E0612F0E94C10286E0602F51
:101280000E94C10287E060E00E94C102E701CC54E5
:10129000DF4F8701025F1E4F85E06D2F0E94C10264
:1012A00086E06C2F0E94C10287E060E00E94C102CC
:1012B0006E96C017D10781F7DF91CF911F910F91E3
:1012C000FF90EF9008951F93CF93DF93E0913B023F
:1012D000F0913C02F7FD12C0CF016AE070E00E947D
:1012E000F117182F16951C5FCF016AE070E00E947D
:1012F000F117C6E8D0E0C61BD10914C02227332756
:101300002E1B3F0BC9016AE070E00E94F117182FF5
:101310001695C9016AE070E00E94F117C62FD0E06F
:10132000C957DF4F80910D0190910E01C817D90761
:1013300039F080910D0190910E010E94240904C0A2
:101340008091BE01811721F0CE01612F0E94D60845
:101350001093BE01D0930E01C0930D01DF91CF9188
:101360001F91089585E060E00E94C10286E06FEC65
:101370000E94C10287E06CE80E94C10285E061E042
:101380000E94C10286E06BE00E94C10287E06DE826
:101390000E94C1020895EF92FF920F931F93CF9383
:1013A000DF937A019EE1699FB0011124680F711DDE
:1013B0008B01020F111D10929503EB0115C085E002
:1013C0006D2F0E94C10286E06C2F0E94C1028091A5
:1013D0009503F701E80FF11D60818F5F80939503FE
:1013E00087E00E94C1022196C017D10740F3DF9128
:1013F000CF911F910F91FF90EF90089581E06EE0E3
:1014000046E051E025E00E94CB090895DF93CF9399
:1014100000D000D0CDB7DEB719821A821C82F894B2
:10142000309143027894832F6AE00E94D117282FCD
:101430000E94D117482F822F0E94D117292F832F66
:101440000E94D117992319F48AE08C8301C09C83F0
:10145000222319F48AE08A8301C02A83498385E420
:101460008B8383E061E0AE014F5F5F4F24E00E9419
:10147000CB090F900F900F900F90CF91DF910895AF
:10148000DF93CF9300D000D0CDB7DEB780E2898361
:101490009BE09A8381E38B839C8381E061E0AE01D2
:1014A0004F5F5F4F21E00E94CB0980918D01813019
:1014B00079F462E0AE014E5F5F4F21E00E94CB09FC
:1014C00081E063E0AE014D5F5F4F22E00E94CB09F7
:1014D0000F900F900F900F90CF91DF910895DF93B1
:1014E000CF9300D000D00F92CDB7DEB7DE011196BA
:1014F000EAE3F1E085E001900D928150E1F78CE0A4
:1015000067E0AE014F5F5F4F25E00E94CB090F906F
:101510000F900F900F900F90CF91DF91089580E082
:101520006CE40E94C1020895809110039091110310
:10153000843B910554F080918B0390E020910E0341
:1015400030910F038217930744F08091BF018823E5
:1015500071F481E08093BF0108958091BF01181656
:1015600024F480E06CE40E94C1021092BF0108954F
:1015700080E062E40E94C10208958F929F92AF9230
:10158000BF92CF92DF92EF92FF920F931F93DF9360
:10159000CF93CDB7DEB72F970FB6F894DEBF0FBE4F
:1015A000CDBFFE013B9685E0DF011D928A95E9F7EC
:1015B00080913F0290914002019797FF02C080E026
:1015C00090E08E010F5F1F4FB8014AE050E00E948B
:1015D000A017F80101900020E9F73197FE2EF01ACC
:1015E00080E0CF2CDD24C7FCD094F6E08F2E912C28
:1015F0008C0E9D1E58010BC0F501E00FF11F80817C
:101600000E94F005080D191DF80180838E2D082F0A
:1016100010E0E82EE3940C151D0574F380939503F8
:1016200085E169E0AE01455F5F4F25E00E94CB098F
:1016300089E18F1969E0A4012F2D0E94CB092F9613
:101640000FB6F894DEBF0FBECDBFCF91DF911F91D3
:101650000F91FF90EF90DF90CF90BF90AF909F9051
:101660008F9008958F929F92AF92BF92CF92DF9208
:10167000EF92FF920F931F93DF93CF93CDB7DEB717
:101680002E970FB6F894DEBF0FBECDBF19821A8217
:101690001B821C828091A8019091A9018E010B5F91
:1016A0001F4FB8014AE050E00E94A017F8010190D6
:1016B0000020E9F73197FE2EF01A80E0CF2CDD24D0
:1016C000C7FCD094AAE08A2E912C8C0E9D1E580146
:1016D0000BC0F501E00FF11F80810E94F005080D9D
:1016E000191DF80180838E2D082F10E0E82EE39459
:1016F0000C151D0574F38093950385E166E0AE013A
:101700004F5F5F4F24E00E94CB0989E18F1966E0AB
:10171000A4012F2D0E94CB098091A8019091A901CD
:101720001816190664F485E060E00E94C10286E0A4
:1017300062EC0E94C10287E06CE80E94C1028091C5
:10174000A8019091A90197FF0CC085E060E00E947C
:10175000C10286E062EC0E94C10287E06DE80E944F
:10176000C1028091A8019091A901892B61F485E0C3
:1017700060E00E94C10286E062EC0E94C10287E044
:1017800060E00E94C1022E960FB6F894DEBF0FBE35
:10179000CDBFCF91DF911F910F91FF90EF90DF9020
:1017A000CF90BF90AF909F908F9008958F929F920F
:1017B000AF92BF92CF92DF92EF92FF920F931F935F
:1017C000DF93CF93CDB7DEB72B970FB6F894DEBF7C
:1017D0000FBECDBFDE011196E7E3F1E083E001909B
:1017E0000D928150E1F78E010C5F1F4F80910C0329
:1017F00090910D03B8014AE050E00E94A017F80153
:1018000001900020E9F73197FE2EF01A80E0CF2CEE
:10181000DD24C7FCD094B8E08B2E912C8C0E9D1E3D
:1018200058010BC0F501E00FF11F80810E94F00507
:10183000080D191DF80180838E2D082F10E0E82E69
:10184000E3940C151D0574F3809395038DE06EE011
:10185000AE014F5F5F4F23E00E94CB0980E18F19FB
:101860006EE0A4012F2D0E94CB092B960FB6F894A1
:10187000DEBF0FBECDBFCF91DF911F910F91FF90C3
:10188000EF90DF90CF90BF90AF909F908F90089592
:101890008F929F92AF92BF92DF92EF92FF920F933F
:1018A0001F93DF93CF93CDB7DEB728970FB6F89489
:1018B000DEBF0FBECDBF19828AE08A8380919A0174
:1018C00090919B018E010D5F1F4FB8014AE050E0DF
:1018D0000E94A017F80101900020E9F73197E01B62
:1018E00080E0EE2EFF24E7FCF094480106E0A02EF5
:1018F000B12CAC0EBD1E0BC0F401E00FF11F8081B6
:101900000E94F0050A0D1B1DF80180838D2D082F04
:1019100010E0D82ED3940E151F0574F38093950311
:1019200080919A0190919B018E010A5F1F4F0A9747
:101930006CF481E06EE0AE014F5F5F4F21E00E94EA
:10194000CB0982E06EE0A80121E004C081E06EE0F6
:10195000A80122E00E94CB0980919C0190919D01F9
:101960008E010D5F1F4FB8014AE050E00E94A017A2
:10197000F80101900020E9F73197E01B80E0EE2E9E
:10198000FF24E7FCF094480116E0A12EB12CAC0E28
:10199000BD1E0BC0F401E00FF11F80810E94F00515
:1019A0000A0D1B1DF80180838D2D082F10E0D82E05
:1019B000D3940E151F0574F38093950380919C01B9
:1019C00090919D018E010A5F1F4F0A976CF484E08D
:1019D0006EE0AE014E5F5F4F21E00E94CB0985E0D3
:1019E0006EE0A80121E004C084E06EE0A80122E0DE
:1019F0000E94CB0928960FB6F894DEBF0FBECDBF6C
:101A0000CF91DF911F910F91FF90EF90DF90BF90EA
:101A1000AF909F908F9008950F931F93DF93CF9374
:101A2000CDB7DEB72A970FB6F894DEBF0FBECDBF95
:101A30008E010F5F1F4FB8014AE050E00E94A017CF
:101A4000F80101900020E9F73197E01B20E0FF2723
:101A5000E7FDF095322F3F5F822F90E08E179F07B2
:101A600014F4232FF7CF209395032A960FB6F894FA
:101A7000DEBF0FBECDBFCF91DF911F910F910895B3
:101A8000AF92BF92CF92DF92EF92FF920F931F938C
:101A9000DF93CF93CDB7DEB76E970FB6F894DEBF66
:101AA0000FBECDBFB82EA62ED42EA42FB52FFD016C
:101AB00001900020E9F73197CE2EC41A7E010894D8
:101AC000E11CF11C242F352FC9018C0108C0F8013D
:101AD00081918F010E94F005F70181937F01802F92
:101AE0008D198C15A0F38B2D6A2DAE014F5F5F4FC2
:101AF0002C2D0E94CB096E960FB6F894DEBF0FBE58
:101B0000CDBFCF91DF911F910F91FF90EF90DF90AC
:101B1000CF90BF90AF90089580918801813061F49B
:101B20008091D00187FD8F5F85958195825F61E00F
:101B300041ED51E00E94400D0895EF92FF920F9306
:101B40001F93DF93CF93CDB7DEB764970FB6F894AA
:101B5000DEBF0FBECDBFF82EE62ECA018E010F5F8D
:101B60001F4FB8014AE050E00E94A0178F2D6E2D44
:101B7000A8010E94400D64960FB6F894DEBF0FBE18
:101B8000CDBFCF91DF911F910F91FF90EF900895FE
:101B9000BF92CF92DF92EF92FF920F931F93DF934A
:101BA000CF93CDB7DEB764970FB6F894DEBF0FBE04
:101BB000CDBFC82EB62EFA017E010894E11CF11C9F
:101BC00004C0AE0DBF1D9C9331968E2F841B949143
:101BD000A82FB0E09923A9F7AE0DBF1D1C92F70105
:101BE00001900020E9F73197DE2EDE18870107C04B
:101BF000F80180810E94F005F80181938F01802F08
:101C00008E198D15A8F38C2D6B2DAE014F5F5F4F94
:101C10002D2D0E94CB0964960FB6F894DEBF0FBE3F
:101C2000CDBFCF91DF911F910F91FF90EF90DF908B
:101C3000CF90BF9008951F93CF93DF93EC01A3E063
:101C4000B0E047C0FD01EC59FD4F8081FD01EB592B
:101C5000FD4F2081422F50E04D535040FD01EA5985
:101C6000FD4F7081FD01E959FD4F10819A01F4E0AB
:101C700035952795FA95E1F790E0CD97880F991F54
:101C8000880F991F282B392B2883613029F1E72FE2
:101C9000F0E0FD9734E0440F551F3A95E1F750709E
:101CA000CF019595879595958795482B592B498315
:101CB000623091F01496635086E0EE0FFF1F8A9514
:101CC000E1F7F070812F90E0CD97E82BF92BEA83B4
:101CD0002396662309F0B6CFDF91CF911F91089527
:101CE000809166028635B1F48091650281568093B9
:101CF000B4018091B401843018F084E08093B40181
:101D00008CE393E06AE043E02AE00E941B0E81E04E
:101D10008093B5011092850108951F931091B4012D
:101D2000123009F48AC0143009F4E2C0113009F00D
:101D30009EC180916602813581F481E793E06BE179
:101D400043E02DE20E941B0E8091710390E090937E
:101D5000B7018093B6011093BA0180916602843472
:101D600009F085C18AEF92E061E443E021E40E943A
:101D70001B0E8091100390911103843B910554F444
:101D800080919401813031F410929401F8940E9472
:101D90004B1078948091100390911103843B91052E
:101DA0007CF080919401882359F481E08093940120
:101DB000F89480918701882311F40E943B10789455
:101DC0008091FC029091FD0266E170E00E94F117A3
:101DD0006E5F7F4F70933E0260933D028091FE02E2
:101DE0009091FF0266E170E00E94F1176A5F7F4FF9
:101DF00070933C0260933B0280910603909107032D
:101E00006EE170E00E94F1177093400260933F0210
:101E100080910E03809343028091220290912302CD
:101E2000909342028093410280912B0290912C0268
:101E300090934602809345021AC1809166028F34C6
:101E4000A9F0813509F013C181E793E06BE143E02C
:101E50002DE20E941B0E8091710390E09093B701D8
:101E60008093B60181E08093BA0101C185EE91E0D3
:101E700060E543E02DE20E941B0E20912D023327E6
:101E800027FD309582E090E0821B930B90933E02F9
:101E900080933D0280912E02992787FD90950696AA
:101EA00090933C0280933B0280912002909121020A
:101EB0009093400280933F028091260280934302D8
:101EC00080912202909123029093420280934102DA
:101ED00080912B0290912C029093460280934502B0
:101EE00080911F028093470281E08093B901BFC0B7
:101EF00080916602843409F056C08AEF92E061E472
:101F000043E021E40E941B0E809110039091110385
:101F1000843B910554F480919401813031F4109206
:101F20009401F8940E944B10789480911003909142
:101F30001103843B91057CF080919401882359F42E
:101F400081E080939401F89480918701882311F4B3
:101F50000E943B1078948091FC029091FD0266E112
:101F600070E00E94F1176E5F7F4F70933E026093A6
:101F70003D028091FE029091FF0266E170E00E94B6
:101F8000F1176A5F7F4F70933C0260933B02809130
:101F90000603909107036EE170E00E94F1177093C1
:101FA000400260933F02809166028C3481F481E0AC
:101FB00090E09093B7018093B60181E08093BA01DD
:101FC00083E793E069E143E02DE20E941B0E8091DC
:101FD00066028D3481F482E090E09093B7018093A3
:101FE000B60181E08093BA0183E793E069E143E0C1
:101FF0002DE20E941B0E809166028E3481F483E0F4
:1020000090E09093B7018093B60181E08093BA018C
:1020100083E793E069E143E02DE20E941B0E80918B
:1020200066028F3481F484E090E09093B70180934E
:10203000B60181E08093BA0183E793E069E143E070
:102040002DE20E941B0E80916602803581F485E0AE
:1020500090E09093B7018093B60181E08093BA013C
:1020600083E793E069E143E02DE20E941B0E1092AA
:1020700085011F91089582E289B910BC80B91CBE08
:10208000909A28E92AB996E890BD82EC8BB921B9DB
:102090009CBF82B9089582E289B910BC80B91CBE88
:1020A00088E98AB926E820BD92EC9BB980E981B91C
:1020B0002CBF92B90895DF93CF93CDB7DEB72C979D
:1020C0000FB6F894DEBF0FBECDBF83E2898383E6EF
:1020D0008A8385E78B838DE38C838D838E838F83C7
:1020E000DE011196FD0120E030E0AE01485F5F4F58
:1020F0008191280F311DE417F507D1F7C9019F70B1
:1021000046E0959587954A95E1F7835C88872F731C
:102110003070822F835C89878DE08A879E01255FDE
:102120003F4F8C91159BFECF83B91196A217B30731
:10213000C1F72C960FB6F894DEBF0FBECDBFCF917E
:10214000DF910895DF93CF93CDB7DEB72C970FB60D
:10215000F894DEBF0FBECDBF8BE189838A8385E50E
:102160008B838AEA8C831D82FE0131969E012A5F51
:102170003F4F8081159BFECF83B93196E217F3075D
:10218000C1F72C960FB6F894DEBF0FBECDBFCF912E
:10219000DF910895DF93CF93CDB7DEB72A970FB6BF
:1021A000F894DEBF0FBECDBF93E299838A836B8321
:1021B000842F86958695835C8C8350E043705070A5
:1021C00064E0440F551F6A95E1F7435C4D838DE34E
:1021D0008E838F83DE011196FD0120E030E0AE0199
:1021E000485F5F4F8191280F311DE417F507D1F744
:1021F000C9019F7056E0959587955A95E1F7835CE4
:1022000088872F733070822F835C89878DE08A875F
:102210009E01255F3F4F8C91159BFECF83B9119690
:10222000A217B307C1F72A960FB6F894DEBF0FBE08
:10223000CDBFCF91DF9108955D9BFECF8DE68CB928
:102240005D9BFECF8FE68CB95D9BFECF89E68CB996
:102250005D9BFECF8EE68CB95D9BFECF8DE08CB989
:102260005D9BFECF8EE38CB90895159BFECF83B99D
:1022700008955D9BFECF8CB90895662359F020E048
:10228000FC01E20FF11DE0815D9BFECFECB92F5FF9
:102290006217B0F708955D9BFECF8EE38CB9089569
:1022A0001F920F920FB60F9211242F933F938F938B
:1022B0009F93AF93BF93EF93FF932CB1209396031B
:1022C00085B398E0892785BB5D9BFECF2CB92D3067
:1022D00059F080917003E82FF0E0E65BFC4F20831B
:1022E0008F5F8093700359C0E0917003F0E0E65B6C
:1022F000FC4F20831092B1011092B2011092B301F1
:1023000030E020E090E03FC02130B9F0213018F0FB
:102310002230C1F524C0A32FB0E0A65BBC4F8C9146
:10232000803211F421E023C0E92FF0E08C91E859CC
:10233000FC4F80839093B10124C0A32FB0E0A65B33
:10234000BC4F8C91803211F422E011C0E92FF0E0F3
:102350008C91E95AFD4F80839093B20112C0A32F54
:10236000B0E0A65BBC4F8C91803219F423E090E082
:1023700009C0E92FF0E08C91E85BFD4F80839093DA
:10238000B3019F5F3F5F80917003831708F0BCCF5C
:1023900081E08093B00110927003FF91EF91BF91A3
:1023A000AF919F918F913F912F910F900FBE0F9002
:1023B0001F9018951F920F920FB60F9211248F93B2
:1023C0009F93EF93FF9393B1909397039D3081F484
:1023D0008091C001813061F4AB981092C00180936C
:1023E0008501E0914703F0E0EC59FD4F90832DC04B
:1023F0008091C001882319F0813039F514C09332DF
:1024000041F480918501882321F481E08093C0010B
:10241000AB9A1092470380914703E82FF0E0EC5904
:10242000FD4F90830CC0E0914703F0E0EC59FD4F65
:10243000908380914703853930F4809147038F5F03
:102440008093470302C01092C001FF91EF919F91CA
:102450008F910F900FBE0F901F90189585B392E04B
:10246000892785BB089590919701913019F485B320
:10247000892785BB08951F920F920FB60F921124E2
:102480002F933F935F936F937F938F939F93AF931C
:10249000BF938091C2019091C301892B81F484B5CF
:1024A00095B59093C9018093C8018EB58F7B8EBD81
:1024B00081E090E09093C3018093C2013AC084B55B
:1024C00095B59093C7018093C6012EB520642EBDAB
:1024D0002091C8013091C9011092C3011092C2012C
:1024E000821B930B865698406CE271E00E94DD17C8
:1024F0007093C5016093C4016730710534F086E0C4
:1025000090E09093C5018093C4012091C401309163
:10251000C50180910201992787FD909528173907F9
:1025200041F0263031052CF42093020181E08093A4
:102530009E01BF91AF919F918F917F916F915F911C
:102540003F912F910F900FBE0F901F901895809183
:10255000B4019091B401813019F0943009F05CC05D
:1025600080910603909107039093A1018093A001AD
:102570008091A0019091A1012091A2013091A3012D
:10258000821B930B9093A5018093A4018091A001DD
:102590009091A1019093A3018093A2014091AC017D
:1025A0005091AD018091A4019091A501E3E0880FC5
:1025B000991FEA95E1F79A0173E0220F331F7A958C
:1025C000E1F7241B350B820F931F68E070E00E9437
:1025D000F1177093AD016093AC012091AE01309181
:1025E000AF014091AC015091AD01C90163E0880F8A
:1025F000991F6A95E1F7821B930B840F951F68E082
:1026000070E00E94F1177093AF016093AE0180916A
:10261000AE019091AF0104C08091410290914202BD
:102620009093A9018093A8010E94320B08958F9284
:102630009F92BF92CF92DF92EF92FF920F931F93E0
:10264000DF93CF93CDB7DEB72B970FB6F894DEBFED
:102650000FBECDBFDE011196E9E4F1E083E0019009
:102660000D928150E1F7809147028E010C5F1F4F60
:1026700090E0B8014AE050E00E94A017F8010190F4
:102680000020E9F73197BE2EB01AEE24FF24CB2CA0
:10269000DD24C7FCD09488E0882E912C8C0E9D1EE2
:1026A0000DC0F801EE0DFF1D80810E94F005F401C0
:1026B000EE0DFF1D80830894E11CF11CEC14FD0459
:1026C00084F388E161E0AE014F5F5F4F23E00E9439
:1026D000CB098BE18B1961E0A4012B2D0E94CB0962
:1026E0002B960FB6F894DEBF0FBECDBFCF91DF9112
:1026F0001F910F91FF90EF90DF90CF90BF909F9030
:102700008F9008958AE161E047E451E022E00E9461
:10271000CB09089583E66FE644E60E94CA10F89458
:1027200028E088E190E00FB6F894A89581BD0FBE2F
:1027300021BDFFCF1F939D991BC18091CA018F5F5F
:102740008093CA0191E09093CC018091CA018530B9
:1027500009F012C18091CE01882309F077C09093CF
:10276000CE011092CF0184E064E00E94C10283E0B8
:1027700061E041ED51E00E94400D83E063E042E101
:1027800052E00E94C80D84E068E00E94C10283E02C
:1027900065E04BE152E00E94C80D8091000181305C
:1027A00029F484E165E04EE352E004C084E165E091
:1027B00041E452E00E94C80D84E060E00E94C10242
:1027C00083E066E04FE152E00E94C80D80918701EE
:1027D000813029F484E166E04EE352E004C084E1F4
:1027E00066E041E452E00E94C80D83E067E045E204
:1027F00052E00E94C80D80918801813029F484E163
:1028000067E04EE352E004C084E167E041E452E057
:102810000E94C80D83E068E04DE252E00E94C80DBE
:1028200080919F01813029F484E168E04EE352E019
:1028300004C084E168E041E452E00E94C80D83E0F6
:102840006BE049E352E00E94C80D94C01091CF01A3
:10285000113049F584E068E00E94C102809187014F
:10286000882339F41093870184E166E04EE352E057
:1028700006C01092870184E166E041E452E00E94C4
:10288000C80D20918701E199FECF80E090E09FBBC9
:102890008EBB2DBB0FB6F894E29AE19A0FBE84E08E
:1028A00060E00E94C1028091CF01823051F584E046
:1028B00068E00E94C10280918801882341F481E090
:1028C0008093880184E167E04EE352E006C01092F5
:1028D000880184E167E041E452E00E94C80D209144
:1028E0008801E199FECF82E090E09FBB8EBB2DBBBB
:1028F0000FB6F894E29AE19A0FBE84E060E00E947D
:10290000C1028091CF01833051F584E068E00E94DC
:10291000C10280919F01882341F481E080939F014F
:1029200084E168E04EE352E006C010929F0184E12A
:1029300068E041E452E00E94C80D20919F01E199B6
:10294000FECF87E190E09FBB8EBB2DBB0FB6F89406
:10295000E29AE19A0FBE84E060E00E94C102809199
:10296000CF01843049F41092CE010E948A1304C032
:102970001092CA011092CC019C99F0C09091CE01A6
:10298000913009F0F1C09093CD018091CB018F5F20
:102990008093CB018091CB01853009F0E5C0109286
:1029A000CB018091CF01823009F466C0833030F4CE
:1029B000882359F0813009F0D7C032C0833009F440
:1029C00086C0843009F0D0C0A3C09093CF0183E0CB
:1029D00065E04BE152E00E94C80D8091000181301A
:1029E00029F484E165E04EE352E004C084E165E04F
:1029F00041E452E00E94C80D84E068E00E94C102F8
:102A000083E066E04FE152E00E94C80D80918701AB
:102A1000813019F484E166E093C084E166E095C0FA
:102A200082E08093CF0183E066E04FE152E00E94B4
:102A3000C80D80918701813029F484E166E04EE37E
:102A400052E004C084E166E041E452E00E94C80D17
:102A500084E068E00E94C10283E067E045E252E062
:102A60000E94C80D80918801813019F484E167E0EB
:102A700067C084E167E069C083E08093CF0167E0CD
:102A800045E252E00E94C80D80918801813029F40E
:102A900084E167E04EE352E004C084E167E041E492
:102AA00052E00E94C80D84E068E00E94C10283E009
:102AB00068E04DE252E00E94C80D80919F01813094
:102AC00019F484E168E03CC084E168E03EC084E041
:102AD0008093CF0183E068E04DE252E00E94C80D90
:102AE00080919F01813029F484E168E04EE352E057
:102AF00004C084E168E041E452E00E94C80D84E033
:102B000068E00E94C10283E06BE049E352E01FC02D
:102B10001092CF0183E06BE049E352E00E94C80DC0
:102B200084E068E00E94C10283E065E04BE152E08E
:102B30000E94C80D80910001813029F484E165E094
:102B40004EE352E004C084E165E041E452E00E94BB
:102B5000C80D84E060E00E94C10206C01092CB0163
:102B60008091CC018091CD011F910895813061F455
:102B7000E199FECF80E090E09FBB8EBB6DBB0FB6AE
:102B8000F894E29AE19A0FBE0895DF93CF93CDB700
:102B9000DEB764970FB6F894DEBF0FBECDBF20E05E
:102BA000BE016F5F7F4F422F50E0E199FECF822F31
:102BB00090E08D5F9F4F9FBB8EBBE09A8DB3FB0172
:102BC000E40FF51F80838823A9F08F3F11F4108252
:102BD00011C02F5FE8CFFD01EF52FE4FA40FB51FCC
:102BE0008C91808311829F5FA92FB0E0A217B30759
:102BF00094F312C0DE011196FD0101900020E9F767
:102C00003197EA1BFB0BE093D00190E02E2F332786
:102C100027FD3095AD01E8CF64960FB6F894DEBF7E
:102C20000FBECDBFCF91DF910895DF93CF93CDB786
:102C3000DEB760970FB6F894DEBF0FBECDBF8091B0
:102C400045029091460290936302809362028091C4
:102C50006202909163026FE070E00E94DD17DE0176
:102C60001596AD016A1B9E01205F3F4FE62FEA0FCC
:102C7000F0E0EC5BFD4FE491ED93A217B307B1F7E1
:102C800019821A821B821C8289E06EE02BE00E946E
:102C9000CB098EE06CE0AE014F5F5F4F24E00E94F5
:102CA000CB0940916202509163028FE06CE00E9478
:102CB0009D0D60960FB6F894DEBF0FBECDBFCF91CD
:102CC000DF910895DF93CF93CDB7DEB7E4970FB6CA
:102CD000F894DEBF0FBECDBFDE011796ECE4F1E045
:102CE00087E001900D928150E1F7DE011E96E3E549
:102CF000F1E089E001900D928150E1F7DE015796F5
:102D0000ECE5F1E08EE001900D928150E1F7DE01FB
:102D10001196EAE6F1E086E001900D928150E1F72C
:102D2000DE019596E0E7F1E080E101900D9281509F
:102D3000E1F7509168036091690340916A038091C3
:102D40006B0320E030E0803711F421E030E080E0D8
:102D500090E04C3611F481E090E02823392380E0A4
:102D6000583609F481E090E0653609F491E0892352
:102D700090E028233923232B79F0CE01079666E0D3
:102D80000E943D11CE010E9668E00E943D11CE01D9
:102D900047966DE00E943D11509168036091690370
:102DA00040916A0380916B0320E030E0873711F493
:102DB00021E030E080E090E04F3611F481E090E0D7
:102DC0002823392380E0533709F481E090E0683606
:102DD00009F491E0892390E028233923232B19F16A
:102DE0008091570290915802893481F4943471F49F
:102DF000CE01019665E00E943D1181ED91E0609168
:102E0000D0010E943D118DE00E943911809157023E
:102E100090915802863739F4953629F4CE0185967B
:102E200068E00E943D118091680320916903409100
:102E30006A0390E0833709F491E080E0253609F4D5
:102E400081E09823892F90E020E030E0443711F4AE
:102E500021E030E082239323892B09F440C0809144
:102E6000570290915802893409F039C0943409F01E
:102E700036C020E01CC0A22FB0E0FD01E85BFD4F92
:102E8000E081E199FECF822F90E08D5F9F4F9FBB45
:102E90008EBBEDBB0FB6F894E29AE19A0FBEFD012E
:102EA000E85BFD4F8081AF52BE4F8C932F5F8091C6
:102EB000B301281700F3E199FECFE22FF0E0CF0134
:102EC0008D5F9F4F9FBB8EBB1DBA0FB6F894E29AE1
:102ED000E19A0FBEEF52FE4F10822093D001509125
:102EE00068036091690340916A0380916B0320E05D
:102EF00030E0853611F421E030E080E090E04337A7
:102F000011F481E090E02823392380E0523709F45E
:102F100081E090E0653609F491E0892390E0282370
:102F20003923232B11F00E948A130E944B11E4963F
:102F30000FB6F894DEBF0FBECDBFCF91DF910895DD
:102F4000FB019F01E8944230C4F04532B4F44A30AA
:102F500029F497FB1EF4909581959F4F642F772756
:102F60000E94DD17805D8A330CF0895D8193CB016F
:102F70000097A1F716F45DE251931082C9010C94F9
:102F8000C117DC01FC01672F71917723E1F73297BC
:102F900004C07C916D9370836291AE17BF07C8F334
:102FA0000895991B79E004C0991F961708F0961BA5
:102FB000881F7A95C9F780950895AA1BBB1B51E11C
:102FC00007C0AA1FBB1FA617B70710F0A61BB70B99
:102FD000881F991F5A95A9F780959095BC01CD013E
:102FE000089597FB092E07260AD077FD04D0E5DF68
:102FF00006D000201AF4709561957F4F0895F6F77A
:0C300000909581959F4F0895F894FFCFA4
:10300C0001010300000A00004400002300230054C7
:10301C0064665363655262005161005060005060F9
:10302C0000516100526200536365546466676869BD
:10303C006A6B6B6A6968670000005353635353FAF9
:10304C0002E50171030D0A0A1D00000068656C7031
:10305C00200D0073686F772049440D0073686F77FB
:10306C002076657273696F6E0D004944203D200017
:10307C00302E392E302E322E622E626574610D0088
:00000001FF
